:100000000C940D060C9454060C9454060C9454064F
:100010000C9454060C9454060C9454060C945406F8
:100020000C9454060C9454060C9445100C9417111F
:100030000C9496200C9454060C9454060C9454067C
:100040000C9454060C94472D0C9454060C945406AE
:100050000C9454060C940A210C9454060C945406E7
:100060000C9454060C9454060C9454060C945406A8
:100070000C9454060C9454060C9454060C94540698
:100080000C9454060C9454060C9454060C94540688
:100090000C9454060C9454060C9454060C94540678
:1000A0000C9454060C9454060C9454062008220810
:1000B00028082D08310836083C083C083C083C0854
:1000C0003C083C083C087F11A2115D12A2115D1290
:1000D000E7110A125D122C123F1297159715C415DD
:1000E000C4151F165916C218C2187116C2186E17F9
:1000F0006E1729183F18C218AE18F1A1F1A1F1A18D
:10010000F1A1351E1F2021222D2E23242526273440
:100110002B141A081517C0C11C180C1213313904FE
:100120001607090A00000B0D0E0F3328E11D1B06F0
:100130001905C2C31110363738E5E0E3E2504F002D
:1001400000000052512F30E4004D2A2C4A29494C1E
:10015000E64B282B4E0001010101010101010101C3
:10016000010101010101010101010101010101017F
:100170000101010101010101000001010101010171
:10018000010101010101010101010101010101015F
:100190000101010000000001010101010001010154
:1001A000010101010101010101000A002530333282
:1001B0006C62003A200025303258000A722F63200A
:1001C000303132333435363738394142434445468D
:1001D0000A000A002530386200626F756E6365217F
:1001E0003A20003D3D3D3D3D3D3D3D3D3D3D3D3D9C
:1001F0003D3D3D3D3D3D3D3D3D3D3D3D0A00536363
:10020000616E3A2025750A003D3D3D3D3D3D3D3D39
:10021000203173207461736B203D3D3D3D3D3D3D7C
:100220003D0A00001080FF000301030203010202E7
:10023000026932632074696D656F75740A00256404
:100240000A0064657461636865640A0061747461BE
:10025000636865640A00657870616E646572207316
:1002600074617475733A202564202E2E2E20005B55
:10027000735D004B6579626F6172642073746172A3
:10028000742E0A0055534220636F6E66696775725B
:1002900065642E0A005B575D005B535D005B525D39
:1002A000005B445D005B435D000A0025303258204E
:1002B000006B6579626F6172645F7265706F7274F2
:1002C0003A20004C45443A20253032580A006465F3
:1002D0006C5F6B65795F6269743A2063616E277445
:1002E0002064656C3A20253032580A006164645FEE
:1002F0006B65795F6269743A2063616E277420616F
:1003000064643A20253032580A00646F6E652E0A04
:1003100000626F6F746D61676963207363616E3A29
:10032000202E2E2E2000290A002575002F0025756D
:10033000005D28002564002000256400200025645D
:100340000020002564007C0025303258006D6F7558
:1003500073656B6579205B62746E7C78207920769A
:1003600020685D287265702F61636C293A205B00FC
:100370006D6B5F776865656C5F74696D655F746FE1
:100380005F6D6178203D2025640A006D6B5F7768A2
:1003900065656C5F6D61785F7370656564203D2095
:1003A00025640A006D6B5F74696D655F746F5F6DC6
:1003B0006178203D2025640A006D6B5F6D61785F78
:1003C0007370656564203D2025640A006D6B5F696C
:1003D0006E74657276616C203D2025640A006D6B39
:1003E0005F64656C6179203D2025640A006D6B5F58
:1003F000776865656C5F74696D655F746F5F6D616B
:1004000078203D2025640A006D6B5F776865656C18
:100410005F6D61785F7370656564203D2025640AB7
:10042000006D6B5F74696D655F746F5F6D617820DF
:100430003D2025640A006D6B5F6D61785F737065A8
:100440006564203D2025640A006D6B5F696E7465EC
:100450007276616C203D2025640A006D6B5F6465D7
:100460006C6179203D2025640A000A00257500365C
:100470003A20776865656C5F74696D655F746F5F5E
:100480006D61783A20000A00257500353A207768BA
:1004900065656C5F6D61785F73706565643A2000B7
:1004A0000A00257500343A2074696D655F746F5FCA
:1004B0006D61783A20000A00257500333A206D619D
:1004C000785F73706565643A20000A002575003214
:1004D0003A20696E74657276616C286D73293A20D2
:1004E000000A00257500313A2064656C6179282A7C
:1004F00031306D73293A20000A092D2056616C7540
:100500006573202D0A004D3E004D25643E20003FBE
:10051000007365742064656661756C740A00433EFF
:10052000200077686572652064656C74613A2063A9
:100530007572736F723D25642C20776865656C3D1C
:1005400025640A53656520687474703A2F2F656EB0
:100550002E77696B6970656469612E6F72672F779A
:10056000696B692F4D6F7573655F6B6579730A00F1
:100570000A092D204D6F7573656B6579202D0A452D
:1005800053432F713A09717569740A313A096465E8
:100590006C6179282A31306D73290A323A09696E03
:1005A00074657276616C286D73290A333A096D613E
:1005B000785F73706565640A343A0974696D655FC4
:1005C000746F5F6D61780A353A09776865656C5FAD
:1005D0006D61785F73706565640A363A097768659E
:1005E000656C5F74696D655F746F5F6D61780A0A31
:1005F000703A097072696E742076616C7565730A61
:10060000643A097365742064656661756C74730A75
:1006100075703A092B310A646F776E3A092D310AE9
:10062000706775703A092B31300A7067646F776EA6
:100630003A092D31300A0A7370656564203D2064E3
:10064000656C7461202A206D61785F7370656564E4
:10065000202A2028726570656174202F2074696DCE
:10066000655F746F5F6D6178290A003F004D3E2021
:1006700000433E20004C25640A000A092D20436FE8
:100680006E736F6C65202D0A4553432F713A0971C3
:100690007569740A6D3A096D6F7573656B65790AD2
:1006A000000A092D204D61676963202D0A643A090B
:1006B00064656275670A783A096465627567206DDA
:1006C00061747269780A6B3A096465627567206BB8
:1006D0006579626F6172640A6D3A09646562756773
:1006E000206D6F7573650A763A0976657273696F66
:1006F0006E0A733A097374617475730A633A096315
:100700006F6E736F6C65206D6F64650A302D343ABF
:10071000096C61796572302D34284631302D4634AC
:10072000290A506175733A09626F6F746C6F616466
:1007300065720A653A09656570726F6D0A6E3A09ED
:100740004E4B524F0A000A002575002E6C657665E7
:100750006C3A20000A002575002E656E61626C659A
:100760003A20000A0025303258006261636B6C69E0
:100770006768745F636F6E6669672E7261773A208F
:10078000000A002575002E6E6B726F3A20000A0079
:100790002575002E737761705F6261636B736C61A6
:1007A00073685F6261636B73706163653A20000A0E
:1007B000002575002E737761705F67726176655FE3
:1007C0006573633A20000A002575002E6E6F5F671F
:1007D00075693A20000A002575002E737761705FF5
:1007E00072616C745F726775693A20000A00257542
:1007F000002E737761705F6C616C745F6C677569F4
:100800003A20000A002575002E636170736C6F63D7
:100810006B5F746F5F636F6E74726F6C3A20000A67
:10082000002575002E737761705F636F6E74726F51
:100830006C5F636170736C6F636B3A20000A002514
:10084000303258006B65796D61705F636F6E6669F9
:10085000672E7261773A20000A002575002E6D6FB1
:100860007573653A20000A002575002E6B65796264
:100870006F6172643A20000A002575002E6D617464
:100880007269783A20000A002575002E656E616253
:100890006C653A20000A00253032580064656275A4
:1008A000675F636F6E6669672E7261773A20000A30
:1008B0000025750064656661756C745F6C617965AF
:1008C000723A20003F004E4B524F3A206F66660A44
:1008D000004E4B524F3A206F6E0A0074696D65727C
:1008E0005F72656164333228293A202530346C58B0
:1008F0000A006B6579626F6172645F6E6B726F3A4A
:100900002025580A006B6579626F6172645F6964C3
:100910006C653A2025580A006B6579626F617264D4
:100920005F70726F746F636F6C3A2025580A0068AD
:100930006F73745F6B6579626F6172645F6C65641D
:100940007328293A2025580A000A092D205374617A
:10095000747573202D0A004743433A20342E392EF4
:1009600032204156522D4C4942433A20312E382EE6
:100970003073766E204156525F415243483A2061AF
:100980007672350A004F5054494F4E533A204C5519
:10099000464120424F4F544D41474943204D4F550A
:1009A00053454B45592045585452414B45592043D6
:1009B0004F4E534F4C4520434F4D4D414E44204EDA
:1009C0004B524F204B45594D41505F494E5F454575
:1009D00050524F4D204C45444D4150204C45444DC4
:1009E00041505F494E5F454550524F4D2042414373
:1009F0004B4C4947485420534F465450574D5F4C39
:100A0000454420425245415448494E475F4C454475
:100A100020343039360A004255494C443A2062624B
:100A20003637336262202831333A32383A3039204F
:100A30005365702031352032303136290A0056494D
:100A4000443A20307831323039284B2E542E452EFE
:100A5000432E29205049443A203078323332382806
:100A60004572676F446F6E6529205645523A2030B3
:100A700078303330310A00444553433A20742E6DA8
:100A80002E6B2E206B6579626F61726420666972CD
:100A90006D7761726520666F72204572676F446F73
:100AA0006E650A000A092D2056657273696F6E2003
:100AB0002D0A000A6D6F7573653A206F66660A002D
:100AC0000A6D6F7573653A206F6E0A000A6B65795F
:100AD000626F6172643A206F66660A000A6B65791C
:100AE000626F6172643A206F6E0A000A6D617472FF
:100AF00069783A206F66660A000A6D6174726978D7
:100B00003A206F6E0A000A64656275673A206F6E5C
:100B10000A000A64656275673A206F66660A000A11
:100B20000A626F6F746C6F616465722E2E2E2000E6
:100B3000433E20006565636F6E6669673A0A000090
:100B40000000000000000000000101010202020399
:100B500003040405050606070808090A0B0B0C0D1B
:100B60000E0F10111213151617191A1B1D1E202215
:100B7000232527292B2D2F313335383A3D3F424449
:100B8000474A4D505356595C5F6266696C70747782
:100B90007B7E82868A8E9195999DA1A5A9ADB0B4E0
:100BA000B8BCC0C3C7CBCED2D5D8DBDFE2E4E7EA1E
:100BB000ECEFF1F3F5F7F8FAFBFCFDFEFFFFFF6247
:100BC00061636B6C6967687420737465703A202583
:100BD000750A006261636B6C6967687420746F6783
:100BE000676C653A2025750A006261636B6C696702
:100BF00068742064656372656173653A2025750ABF
:100C0000006261636B6C6967687420696E6372650A
:100C10006173653A2025750A000011241FBECFEFCD
:100C2000DAE0DEBFCDBF04B603FE27C080916C04BE
:100C300090916D04A0916E04B0916F048730904B39
:100C4000A740B04BD1F410926C0410926D04109236
:100C50006E0410926F0414BE84B7877F84BF0FB6F2
:100C6000F894A8958091600088618093600010924C
:100C700060000FBEE0E0F8E3099513E0A0E0B1E00A
:100C8000E6E5F8E602C005900D92AA32B107D9F761
:100C900024E0AAE2B3E001C01D92AC36B207E1F74E
:100CA0000E94FF0D0C9429340C940000FF93EF93E5
:100CB000E0912A03F0912B03309709F00995EF9109
:100CC000FF910895FC018591803011F0EFDFFBCF9B
:100CD0000895FF27E0E230E247FF0CC0419597FFFF
:100CE00009C0EDE26095709580959095611D711D2C
:100CF000811D911D27FF02C0219530E350E2AA27F4
:100D0000660F771F881F991FAA1FA41710F0A41B36
:100D100063955A95A9F7AA3008F0A95FA05DAF9333
:100D2000F395611571058105910541F7ED3211F4D7
:100D3000EF93F395F21718F43F93F395FBCF8F9150
:100D4000B5DFFA95E1F70895E991F9918591803041
:100D500021F0853219F0AADFF9CF089520E0E89458
:100D600055915532C1F3503311F4689455915A336B
:100D700048F4505390F3220F022E220F220F200D21
:100D8000250FF4CF0EF4219589919991533619F3DB
:100D9000533729F1533559F1BC0188279927E89435
:100DA0005C3621F48991999168945591543639F4BF
:100DB00046EF7EF077FF0DC08FEF9FEF0AC05537EB
:100DC0004AE039F0583540E121F0523642E009F06E
:100DD0000895FF93EF937DDFEF91FF91B7CFFF93DE
:100DE000EF93FC0181918030B9F360DFFBCFFF937B
:100DF000EF9368DFF1CFDF93CF93CDB7DEB72596C2
:100E0000A3DFCF91DF91089588EA90E0089584E010
:100E100090E00895462F672F0C94D731805C0E9494
:100E2000CB31089582E091E008958AEF90E0089533
:100E300080B38F7080BB81B38F7081BB84B1897F99
:100E400084B985B1897F85B90C94DC0A86E0089560
:100E50008EE00895EF92FF920F931F93CF93DF934D
:100E600080E885BF85BF0E94BF208FE99FE0019782
:100E7000F1F700C000000E94C82090932D038093DA
:100E80002C030E9418076E98769A8AB183768AB9E5
:100E90008BB18C698BB93E98469A24982C9A0E9403
:100EA0004D0BCFE8D3E082E8E82E83E0F82E0EE287
:100EB00013E01992199210928E030E94C820F70134
:100EC000819391937F0180E090E0F801E80FF91F92
:100ED000108201968E309105C1F7025F1F4FF3E03B
:100EE000CB39DF0731F7DF91CF911F910F91FF9041
:100EF000EF9008958F929F92AF92BF92CF92DF9220
:100F0000EF92FF920F931F93CF93DF9380912C0367
:100F100090912D030E94E020883E9340A0F18091A3
:100F20001B0480FF08C088E092E09F938F930E948B
:100F3000FB060F900F9080911B0480FF10C08091E2
:100F40002D038F9380912C038F938EEF91E09F93CD
:100F50008F930E94FB060F900F900F900F900E94AE
:100F6000C82090932D0380932C030E94F70A809150
:100F70001B0480FF08C083EE91E09F938F930E9433
:100F8000FB060F900F90E0918E03F0E0EE0FFF1F35
:100F9000EE57FC4F808191810E94E0205C01892BFB
:100FA00009F4FEC0C0918E03D0E00E94C820CC0F8F
:100FB000DD1FCE57DC4F9983888380918E0382306A
:100FC00099F038F4882369F08130B1F4859A8D98CE
:100FD00013C0843079F058F0853071F4229A2A9841
:100FE0000BC0849A8C9808C0869A8E9805C0879A00
:100FF0008F9802C0219A29980E94E00A80EA8A9577
:10100000F1F70E94790BC0E0D0E0BB24B3942DE04F
:10101000822E3EE0932EEE24E394F12C04ED11E0B9
:10102000C0908E03D12C8C2F90E0FC013197ED30D5
:10103000F10520F4EA5AFF4F0C94DE3383B10EC061
:101040008CB107C089B18095881F8827881F18C078
:1010500086B186FB882780F90DC089B182958170A1
:1010600009C089B182FB882780F904C089B183FB5C
:10107000882780F98B2504C0882D8C1B0E94A70A25
:101080002A2D9C9CF0019D9CF00D1124EC0FFD1F5E
:10109000E25DFC4F9081990F982B2150E1F79C9CC9
:1010A000F0019D9CF00D1124EC0FFD1FE25DFC4F43
:1010B0009083E0918E03F0E097010C2E02C0220F86
:1010C000331F0A94E2F7892F8F718F30C9F040F4F3
:1010D0008130B1F018F1833099F0873089F510C074
:1010E0008C3109F456C038F4803109F452C088318B
:1010F00009F44FC025C08E3109F44BC08F3101F582
:10110000EE0FFF1FE157FC4F80819181A901482319
:101110005923452BF1F5282B392B0FC0EE0FFF1F5C
:10112000E157FC4F80819181A90148235923452B28
:1011300081F120953095282339233183208329C0DC
:1011400080911B0480FF04C089ED91E00E9462063B
:1011500080911B0480FF15C09C9CF0019D9CF00DAC
:101160001124EC0FFD1FE25DFC4F80818F711F92F7
:101170008F931F930F930E94FB060F900F900F9079
:101180000F9080911B0480FF04C082ED91E00E94CB
:1011900062062196CE30D10509F042CF0E94180791
:1011A00080918E038F5F863018F480938E0302C087
:1011B00010928E0381E0DF91CF911F910F91FF90EC
:1011C000EF90DF90CF90BF90AF909F908F90089559
:1011D000E82FF0E0EE0FFF1FE157FC4F8081918177
:1011E0000895CF92DF92EF92FF920F931F93CF93C8
:1011F000DF938BEB91E00E9462068FE8E82E83E09C
:10120000F82EC0E0D0E096EBC92E91E0D92E0CEA82
:1012100011E0DF93CF93DF92CF920E94FB0683EB26
:1012200091E00E946206F701619171917F0180E077
:1012300090E00E9414209F938F937F936F931F934E
:101240000F930E94FB068AEA91E00E9462062196B3
:101250008DB79EB70A960FB6F8949EBF0FBE8DBF8E
:10126000C630D105B1F6DF91CF911F910F91FF905C
:10127000EF90DF90CF900895CF93C82F0E94AC2CB1
:10128000C730A0F4C430F0F4C130A0F10E94CA2CE1
:101290000E940D2D0E94412DEC2FF0E0ED5DFD4FE1
:1012A000849180935D04CF910C94DF2CC730A9F01A
:1012B000C83001F50E94CA2C0E94072D0E94412DC2
:1012C00081E012C00E94CA2C0E940D2D0E943B2D6D
:1012D00086E08C1BCF910C94442D0E94CA2C0E9456
:1012E000072D0E94412D80E00E942A2D83E0CF919E
:1012F0000C94382D0E940D2D0E94412D10925D04FA
:1013000080E00E94DF2CCF910C94D02CE82FF0E0ED
:10131000EE0FFF1FE95DFD4F85919491089584B113
:10132000886684B985B1877985B9209A289A559AB3
:101330005D9A0895823079F028F4882341F0813055
:1013400041F00895833049F0843049F008952D9A92
:1013500008952E9A08952B9A0895289808955D98D7
:101360000895823079F028F4882341F0813041F0EB
:101370000895833049F0843049F008952D980895F8
:101380002E9808952B980895289A08955D9A0895A7
:1013900081E392E09F938F930E94FB061092BC0022
:1013A000509A519880EA8A95F1F70F900F90499BD7
:1013B00005C0509884E98093BC00089589E058984E
:1013C00095E09A95F1F70000589A95E09A95F1F713
:1013D00000008150A1F7EDCF1092B9008CE080930E
:1013E000B80008951F93CF93DF93182F84EA80935A
:1013F000BC0091E08091BC0087FD12C0992321F0D0
:101400000E94C820EC010AC0CE010E94E020883B67
:101410009B4020F00E94C80982E02BC090E0EACFF8
:101420009091B900987F983021F0903111F081E0CF
:1014300020C01093BB0084E88093BC0081E09091B1
:10144000BC0097FD0EC0882321F00E94C820EC014B
:1014500006C0CE010E94E020883B9B40D8F680E089
:10146000EECF8091B900887F883111F08034F9F691
:1014700080E0DF91CF911F9108950C94F209CF93F2
:10148000DF9384E98093BC0091E02091BC0024FFAD
:1014900012C0992321F00E94C820EC010AC0CE019D
:1014A0000E94E020883B9B4020F0DF91CF910C947C
:1014B000C80990E0EACFDF91CF910895CF93DF93F1
:1014C0008093BB0084E88093BC0091E02091BC0035
:1014D00027FD12C0992321F00E94C820EC010AC008
:1014E000CE010E94E020883B9B4020F00E94C8096A
:1014F00082E009C090E0EACF9091B900987F81E046
:10150000983209F480E0DF91CF910895CF93DF9373
:1015100084E88093BC0091E02091BC0027FD12C0BC
:10152000992321F00E94C820EC010AC0CE010E943C
:10153000E020883B9B4020F00E94C80982E004C064
:1015400090E0EACF8091BB00DF91CF910895853084
:1015500008F08F5F20919B0330E0A90102C05595F0
:1015600047958A95E2F7CA01817008950F931F93FA
:10157000CF93DF931F92CDB7DEB790919C03992351
:10158000A1F0062F182F80E40E94F209811108C0F3
:10159000812F0E945E0A811103C0802F0E945E0A83
:1015A00089830E943F0A8981982F892F0F90DF91AC
:1015B000CF911F910F9108956FEF81E00C94B60ABF
:1015C0008F5F61E070E001C0660F8A95EAF7609571
:1015D00081E00C94B60A6FEF82E00E94B60A6FEFCA
:1015E0008CE00E94B60A6FEF81E00C94B60A8091FD
:1015F0001B0480FF0EC080919C031F928F9386E591
:1016000092E09F938F930E94FB060F900F900F9094
:101610000F9080E40E94F209811118C00E943F0AD5
:1016200080919C03811126C080911B0480FF08C01B
:101630008CE492E09F938F930E94FB060F900F9093
:1016400081E080939C030E94EB0A12C080919C036E
:10165000813081F480911B0480FF08C082E492E015
:101660009F938F930E94FB060F900F9010929C0304
:101670000E94E31880911B0480FF0EC080919C03A0
:101680001F928F938EE392E09F938F930E94FB06AD
:101690000F900F900F900F9008950E94EC090C94FA
:1016A000F70A0F931F93CF93DF93C0919C03CC2332
:1016B000D1F08B01D82F80E40E94F209C82F81114C
:1016C00010C08D2F0E945E0AC82F81110AC081E4CC
:1016D0000E943D0AC82F811104C00E94860AF801A9
:1016E00080830E943F0A8C2FDF91CF911F910F9131
:1016F00008956BE973E082E10C94510B8091B00383
:1017000008959FB7F89410929F039FBF9091610432
:10171000943009F057C09091E9009F703091EC002F
:10172000232F217030FD20E8922B24E02093E90044
:101730002091EB0020FF43C02091EE0027FF3FC027
:1017400020919D03222321F02091E80025FF37C03E
:1017500010929D0326E03091E80035FD15C03091D0
:101760006104343061F53091EB0035FD28C0215023
:1017700021F481E080939D0322C0EFE9FFE03197DF
:10178000F1F700C00000E7CF8093F1008091E800FE
:1017900085FD0AC08091E80080FFFCCF8091E800C1
:1017A0008E778093E80006C08FB7F89421E02093ED
:1017B0009F038FBF9F709093E90080E008959F7012
:1017C0009093E9008FEF0895CF93DF9300D01F929D
:1017D000CDB7DEB79C0180916104843019F593E0A8
:1017E00099833B832A839093E9008FEF9091E800DF
:1017F000815095FD06C095ED9A95F1F70000811195
:10180000F5CF8091E80085FF0DC040E050E063E037
:1018100070E0CE0101960E94B90E8091E8008E77AB
:101820008093E8000F900F900F90DF91CF91089573
:10183000CF93DF9300D01F92CDB7DEB72091610424
:10184000243021F522E029839B838A8383E08093DF
:10185000E9008FEF9091E800815095FD06C095ED6D
:101860009A95F1F700008111F5CF8091E80085FF8E
:101870000DC040E050E063E070E0CE0101960E94B0
:10188000B90E8091E8008E778093E8000F900F905A
:101890000F90DF91CF910895209161042430F1F4ED
:1018A00022E02093E9002FEF3091E800215035FD30
:1018B00006C035ED3A95F1F700002111F5CF2091E2
:1018C000E80025FF0BC040E050E065E070E00E94BA
:1018D000B90E8091E8008E778093E8000895CF9349
:1018E000DF9320916104243009F048C0EC0180911D
:1018F0000A018823E1F080910B018823C1F085E083
:101900008093E9008FEF9091E800815095FD06C02B
:1019100095E19A95F1F700008111F5CF8091E800EB
:1019200085FF2CC040E050E060E170E017C081E02E
:101930008093E9008FEF9091E800815095FD06C0FB
:1019400095ED9A95F1F700008111F5CF8091E800AF
:1019500085FF14C040E050E068E070E0CE010E94D6
:10196000B90E8091E8008E778093E80080E1FE0157
:10197000A0EAB3E001900D928A95E1F7DF91CF9153
:10198000089585EA92E00E946206809160048111C8
:1019900009C00E94CC0F0E9427108091E200846051
:1019A0008093E200089581EA92E00E94620610921C
:1019B000600408958DE992E00C94620620919E03E4
:1019C0002F5F822F62E30E94BE33992319F0209388
:1019D0009E03089510929E0380919F03882371F1C6
:1019E00080916104843041F58091E9008F702091ED
:1019F000EC00922F917020FD90E8892B94E0909359
:101A0000E9009091EB0090FF14C09091EE0097FFD9
:101A100010C09091E80095FF03C01092F100F9CF3B
:101A20009091E80090FF05C09091E8009E77909318
:101A3000E8008F708093E90010929F03089542E0C0
:101A400061EC81E00E94670F42E061EC82E00E945D
:101A5000670F42E061EC83E00E94670F42E261ECB5
:101A600084E00E94670F42E161EC85E00C94670F0F
:101A700080916304833009F455C030F4813071F0F3
:101A8000823009F48EC008958A3009F47AC08B3010
:101A900009F460C0893009F09CC020C080916204C4
:101AA000813A09F096C08091E800877F8093E80032
:101AB0008091660490916704892B21F460E180EAAB
:101AC00093E003C060E080E090E070E00E94040FCB
:101AD0008091E8008B778093E800089580916204FC
:101AE000813209F076C08091660490916704009776
:101AF00019F0049709F06DC08091E800877F80930A
:101B0000E8008091E80082FD05C0809161048111A8
:101B1000F8CF5FC08091F1008093B0038091E8001E
:101B20008B7753C080916204813A09F052C0809152
:101B3000660490916704892B09F04BC08091E800FE
:101B4000877F8093E8008091E80080FFFCCF809140
:101B50000A0136C0809162048132D9F58091660411
:101B600090916704892BA9F58091E800877F809385
:101B7000E8000E947B0F8091640480930A010C941A
:101B8000E31880916204813221F58091E800877F1B
:101B90008093E8000E947B0F809165048093B103DD
:101BA000089580916204813AA1F48091E800877FD2
:101BB0008093E8008091E80080FFFCCF8091B10322
:101BC0008093F1008091E8008E778093E8000C9478
:101BD0007B0F089508950895089589E992E00E9481
:101BE00062060C94EC0D0E94502080915F048823C3
:101BF00029F00E947D2081110C94A30E089584B7D2
:101C0000877F84BF0FB6F894A895809160008861A3
:101C100080936000109260000FBE90E080E80FB6E5
:101C2000F89480936100909361000FBE0E94EA0DCA
:101C30000E9403130E94CC0F0E9427108091E200A3
:101C400084608093E20081E89BE00E94DF1F78942B
:101C5000809161048430E1F784E892E00E9462069A
:101C60000E94051380E091E00E94711283E792E0E8
:101C70000E9462060E94EB0D80916104853039F468
:101C80008FE692E00E9462060E94F30DF5CF0E945B
:101C90001513F2CF0C94922085E992E00E9462061F
:101CA0000C944A0E292F332723303105C1F05CF400
:101CB0002130310579F022303105E9F58DE890E0E9
:101CC00022E631E03CC021323105C1F0223231053B
:101CD00011F131C082E190E02FEE31E030C0992760
:101CE0008330910540F5FC01EE0FFF1FE05DFE4FD4
:101CF00020813181FC01E35DFE4F1AC06530D8F4CC
:101D0000E62FF0E0EE0FFF1FED5DFE4F20813181E9
:101D100089E090E014C0653070F470E0FB01EE0FD4
:101D2000FF1FE75EFE4F20813181FB01EC5EFE4F1D
:101D3000808190E004C080E090E020E030E0FA0193
:101D400031832083089580E189BD82E189BD09B492
:101D500000FEFDCF8091D8008F7D8093D8008091C8
:101D6000E00082608093E0008091E00081FDFCCF84
:101D70000895CF92DF92EF92FF920F931F93CF932C
:101D8000DF93EC018B016A010E949A0F811133C02D
:101D9000C114D10439F0F60180819181081B190B1F
:101DA000C80FD91FE12CF12C0115110519F18091F3
:101DB000E80085FD16C08091E8008E778093E800EA
:101DC000C114D10449F0F60180819181E80EF91E19
:101DD000F182E08285E00FC00E949A0F882321F3F0
:101DE0000AC089918093F10001501109FFEFEF1AA9
:101DF000FF0ADACF80E0DF91CF911F910F91FF9022
:101E0000EF90DF90CF90089520916804309169049D
:101E10002617370748F06115710539F42091E8005D
:101E20002E772093E80001C0B90140E061157105EB
:101E3000A9F120916104222309F443C0253009F45B
:101E400042C02091E80023FD40C02091E80022FD1F
:101E500032C02091E80020FFE9CF4091F3002091AB
:101E6000F20030E0342BFC01CF016115710559F00F
:101E70002830310540F481918093F100615071095F
:101E80002F5F3F4FF1CF41E02830310509F040E0AE
:101E90002091E8002E772093E800C8CF4111C9CFE8
:101EA0000AC080916104882361F0853061F08091DF
:101EB000E80083FD0AC08091E80082FFF2CF80E055
:101EC000089582E0089583E0089581E008958F7079
:101ED0008093E900EBEEF0E0808181608083EDEE9D
:101EE000F0E010826093EC0040838091EE00881F48
:101EF0008827881F08958091620487FF11C0809110
:101F0000E80082FD05C0809161048111F8CF11C005
:101F10008091E8008B770BC080916104882349F0A1
:101F20008091E80080FFF8CF8091E8008E77809361
:101F3000E80008952091E4003091E50095E6409195
:101F4000EC00842F817040FF22C08091E80080FD6A
:101F50001CC080916104882391F0853091F08091BC
:101F6000EB0085FD10C04091E4005091E500421760
:101F7000530729F39A01915011F784E0089582E004
:101F8000089583E0089581E0089580E008954091E8
:101F9000E80042FFDECF08950E9438100E944010F2
:101FA000E0EEF0E0808181608083E8EDF0E0808108
:101FB0008F77808319BCA7EDB0E08C918E7F8C93D6
:101FC00080818F7E80831092600408950F931F9309
:101FD000CF93DF930E9438100E944010C8EDD0E0EC
:101FE00088818F77888388818068888388818F7DC6
:101FF000888319BC1092610410925E0410925F04F1
:1020000000EE10E0F80180818B7F80838881816001
:10201000888342E060E080E00E94670FE1EEF0E03C
:1020200080818E7F8083E2EEF0E08081816080831A
:10203000808188608083F80180818E7F80838881A1
:1020400080618883DF91CF911F910F910895E8ED12
:10205000F0E080818F7E8083E7EDF0E08081816019
:10206000808384E082BF81E0809360040C94E60F5B
:10207000E8EDF0E080818E7F80831092E200089589
:102080001092DA001092E10008951F920F920FB69D
:102090000F9211242F933F934F935F936F937F93EE
:1020A0008F939F93AF93BF93EF93FF938091E10042
:1020B00082FF0BC08091E20082FF07C08091E100A7
:1020C0008B7F8093E1000E94DE0C8091DA0080FF1C
:1020D0001FC08091D80080FF1BC08091DA008E7FE6
:1020E0008093DA008091D90080FF0DC080E189BD26
:1020F00082E189BD09B400FEFDCF81E080936104D7
:102100000E94C10C05C019BC109261040E94D30C3E
:102110008091E10080FF19C08091E20080FF15C02E
:102120008091E2008E7F8093E2008091E2008061E6
:102130008093E2008091D80080628093D80019BC1F
:1021400085E0809361040E94ED0D8091E10084FFA1
:1021500030C08091E20084FF2CC080E189BD82E123
:1021600089BD09B400FEFDCF8091D8008F7D80939A
:10217000D8008091E1008F7E8093E1008091E200A1
:102180008F7E8093E2008091E20081608093E20084
:1021900080915E04882311F084E007C08091E30001
:1021A00087FD02C081E001C083E0809361040E944A
:1021B0004C0E8091E10083FF29C08091E20083FFF3
:1021C00025C08091E100877F8093E10082E08093C9
:1021D000610410925E048091E1008E7F8093E100A3
:1021E0008091E2008E7F8093E2008091E200806126
:1021F0008093E20042E060E080E00E94670F8091FF
:10220000F00088608093F0000E94DA0CFF91EF915B
:10221000BF91AF919F918F917F916F915F914F91FE
:102220003F912F910F900FBE0F901F9018951F9206
:102230000F920FB60F9211242F933F934F935F93FA
:102240006F937F938F939F93AF93BF93CF93DF93BE
:10225000EF93FF93C091E900CF708091EC00D82FED
:10226000D17080FDD0E81092E9008091F000877F66
:102270008093F00078940E945B111092E9008091A5
:10228000F00088608093F000CD2BCF70C093E90000
:10229000FF91EF91DF91CF91BF91AF919F918F917E
:1022A0007F916F915F914F913F912F910F900FBE52
:1022B0000F901F9018951F93CF93DF9300D0CDB749
:1022C000DEB7E2E6F4E088E08E0F9091F1009193A2
:1022D0008E13FBCF0E94380D8091E80083FFEDC084
:1022E0008091620490916304492F50E04A30510577
:1022F00008F0E3C0FA01ED59FF4F0C94DE3380384B
:1023000081F0823809F0D9C0809166048F70809383
:10231000E9008091EB0085FB882780F91092E900A5
:1023200007C080915F04882311F082E001C080E043
:102330009091E800977F9093E8008093F1001092CD
:10234000F10095C0282F2D7F09F0B7C0882319F020
:10235000823061F0B2C080916404813009F0ADC078
:10236000933009F080E080935F042BC08091640477
:10237000811127C0809166048F7009F49EC08093FC
:10238000E9002091EB0020FF1CC0933021F48091E4
:10239000EB00806214C09091EB0090619093EB0091
:1023A00021E030E0A90102C0440F551F8A95E2F7F1
:1023B0004093EA001092EA008091EB0088608093DD
:1023C000EB001092E9008091E800877F53C08111F3
:1023D00074C0109164041F778091E3008078812B92
:1023E0008093E3008091E800877F8093E8000E945B
:1023F0007B0F8091E80080FFFCCF8091E300806834
:102400008093E300111102C082E001C083E0809359
:10241000610453C08058823008F04FC0AE014F5F56
:102420005F4F6091660480916404909165040E94FE
:10243000520EBC01892B09F440C09091E800977FAF
:102440009093E80089819A810E94040F8091E800AE
:102450008B778093E80031C0803879F58091E8006F
:10246000877F8093E80080915E048093F1008091E3
:10247000E8008E778093E8000E947B0F1EC08111D8
:102480001CC0909164049230C0F48091E800877F72
:102490008093E80090935E040E947B0F80915E041D
:1024A000811106C08091E30087FD02C081E001C078
:1024B00084E0809361040E941F0D8091E80083FFF7
:1024C0000AC08091E800877F8093E8008091EB004C
:1024D00080628093EB000F900F90DF91CF911F915E
:1024E00008959093B7038093B6030895E091B603DF
:1024F000F091B703309721F00190F081E02D09941D
:1025000080E00895EF92FF920F931F93CF93DF9394
:10251000E091B603F091B7033097B1F18C010280DE
:10252000F381E02D099580911B0482FF2DC080FF6F
:1025300004C081EB92E00E946206E80110E18BEAA0
:10254000E82E82E0F82E80911B0480FF0BC088816A
:102550001F928F93FF92EF920E94FB060F900F90B5
:102560000F900F90115021961111EDCF80911B0407
:1025700080FF0AC089EA92E0DF91CF911F910F910D
:10258000FF90EF900C946206DF91CF911F910F9115
:10259000FF90EF900895E091B603F091B703309764
:1025A00021F00480F581E02D099408952091B40371
:1025B0003091B5038217930771F09093B503809320
:1025C000B403E091B603F091B703309721F0068091
:1025D000F781E02D099408952091B2033091B3035F
:1025E0008217930771F09093B3038093B203E09145
:1025F000B603F091B703309721F00084F185E02D08
:102600000994089508950C9402130E94BF200E941B
:102610002A070E94E1220E942F310E94992F0E94D6
:10262000992C0E945E2E0C9486324F925F927F927C
:102630008F929F92AF92BF92CF92DF92EF92FF92D2
:102640000F931F93CF93DF9300D000D01F92CDB78D
:10265000DEB70E947A0799EBC92E93E0D92E00E0ED
:1026600010E0AA24A394B12C702E802F0E94E808B9
:102670004C01F601419051906F01482659264114B2
:102680005104B1F40F5F1F4F0630110569F78FEF4A
:1026900089838A831B820E94C8208160782F9D8352
:1026A0008C8349815A816B818D810E94E61341C0E0
:1026B00080911B0481FD0E94F10820E030E075014B
:1026C000022E02C0EE0CFF1C0A94E2F7C70184211F
:1026D0009521892B41F129837A828E209F2091E0D8
:1026E000892809F490E09B830E94C8208160782F9C
:1026F0009D838C8349815A816B818D810E94E61371
:1027000049815A816B817C818D810E944020000F1C
:10271000111FF801E754FC4F80819181E826F926CA
:10272000F182E08206C02F5F3F4F2E30310539F62F
:10273000A9CF0E943F200E9486261091B8030E94D4
:102740007612181771F10E9476128093B803909157
:102750001B0492FF0EC090FF0CC01F928F9383EC5E
:1027600092E09F938F930E94FB060F900F900F9023
:102770000F908091B8030F900F900F900F900F90D3
:10278000DF91CF911F910F91FF90EF90DF90CF904D
:10279000BF90AF909F908F907F905F904F900C94E0
:1027A000FB2F0F900F900F900F900F90DF91CF9114
:1027B0001F910F91FF90EF90DF90CF90BF90AF905F
:1027C0009F908F907F905F904F900895CF93DF936D
:1027D000CDB7DEB72B970FB6F894DEBF0FBECDBFD7
:1027E000942F4F83252F588769877A878B874A854F
:1027F0005B85452B21F02F3F09F59F3FF9F4DE0162
:10280000119686E0FD0111928A95E9F785E0FE01B7
:10281000379601900D928A95E1F749815A816B8133
:102820007C818D819E810E947D1B2B960FB6F89432
:10283000DEBF0FBECDBFDF91CF9108954F81588588
:1028400069857A858B850E944020D9CFCF938823D4
:1028500009F4CDC0C82F823859F40E94761281FD48
:10286000C6C089E30E94081E0E94B91F89E30CC0FC
:10287000833879F40E94761280FDB9C083E50E9406
:10288000081E0E94B91F83E50E94DC1ECF910C94A4
:10289000B91F843859F40E94761282FDA8C087E4DB
:1028A0000E94081E0E94B91F87E4EECF8CEF8C0FA8
:1028B000813A48F48C2F0E94442B811198C08C2FB0
:1028C0000E94081EE3CF80E28C0F883048F4C77066
:1028D00081E001C0880FCA95EAF70E94881FD6CF11
:1028E0008BE58C0F833078F4C53A29F0C63A31F085
:1028F00083E890E005C081E890E002C082E890E0C3
:10290000CF910C94D61288E58C0F853108F06FC0FA
:10291000C83A61F1C93A69F1CA3A71F1CB3A79F131
:10292000CC3A81F1CD3A89F1CE3A91F1CF3A99F191
:10293000C13BA1F1C03BA9F1C23BB1F1C33BB9F12D
:10294000C43BC1F1C53BC9F1C63BD1F1C73BD9F18D
:10295000C83BE1F1C93BE9F1CA3BF1F1CB3BF9F1ED
:10296000CC3B09F43FC080E090E03EC082EE90E0B6
:102970003BC089EE90E038C08AEE90E035C085EB30
:1029800090E032C086EB90E02FC083EB90E02CC04B
:1029900084EB90E029C087EB90E026C08CEC90E0BF
:1029A00023C08DEC90E020C083E891E01DC08AE850
:1029B00091E01AC082E991E017C084E991E014C067
:1029C00081E292E011C083E292E00EC084E292E0E4
:1029D0000BC085E292E008C086E292E005C087E283
:1029E00092E002C08AE292E0CF910C94EC12CF9177
:1029F0000895882309F44BC0823859F40E94761256
:102A000081FF45C089E30E94081E0E94B91F89E327
:102A10000CC0833871F40E94761280FF38C083E5C1
:102A20000E94081E0E94B91F83E50E94DC1E0C94C0
:102A3000B91F843859F40E94761282FF28C087E4B7
:102A40000E94081E0E94B91F87E4EFCF9CEF980FE9
:102A5000913A58F390E2980F983050F4877091E0D3
:102A600001C0990F8A95EAF7892F0E948E1FDFCF48
:102A70009BE5980F933020F480E090E00C94D61200
:102A8000885A853120F480E090E00C94EC1208958F
:102A9000882321F00E94881F0C94B91F0895882371
:102AA00021F00E948E1F0C94B91F0895CF92DF92DF
:102AB000EF92FF920F931F93CF93DF93CDB7DEB7C3
:102AC00027970FB6F894DEBF0FBECDBF25E0FC01FF
:102AD000DE01119601900D922A95E1F7FC014081EB
:102AE00031810281258122952F7063817481672B4A
:102AF00009F448C33F3F19F44F3F09F443C36C0145
:102B000049833A8389819A812F830E94C71D182F98
:102B10009E830E94C61D0E94D61C9E81E92FE295CD
:102B2000EF70F0E0E359FF4F2F810C94DE33892FD3
:102B3000807F9F70F92E882319F0F29490EFF9228C
:102B4000002349F0FF2009F45FC28F2D0E949B1FD4
:102B50000E94B91F59C2812F0E94F914FF2009F465
:102B600011C38F2D0E94A11F27960FB6F894DEBFC8
:102B70000FBECDBFDF91CF911F910F91FF90EF90CE
:102B8000DF90CF900C94B91F892F807F9F70F92E12
:102B9000803219F0F29480EFF822112319F01130ED
:102BA00001F129C00023A9F08F2D222349F1213002
:102BB00039F527960FB6F894DEBF0FBECDBFDF9173
:102BC000CF911F910F91FF90EF90DF90CF900C94D9
:102BD000AB1F222319F0213009F4D4C20E94AE1F8A
:102BE0002CC00023E9F0263008F0CCC20E94851FDB
:102BF0008F2129F022C00023F1F0211115C08F2D63
:102C000027960FB6F894DEBF0FBECDBFDF91CF91F0
:102C10001F910F91FF90EF90DF90CF900C9448158B
:102C2000253008F0AFC209C0F601858180FFECC1F4
:102C30008F708583E4CF2111FBC18F2D69C1292FAE
:102C400026952695237030E02115310521F021309D
:102C50003105C1F097C2002319F0812F937002C093
:102C600080E090E027960FB6F894DEBF0FBECDBF90
:102C7000DF91CF911F910F91FF90EF90DF90CF9058
:102C80000C94D612002319F0812F937002C080E0BB
:102C900090E027960FB6F894DEBF0FBECDBFDF9150
:102CA000CF911F910F91FF90EF90DF90CF900C94F8
:102CB000EC12812F002319F00E940C2502C00E9403
:102CC000742527960FB6F894DEBF0FBECDBFDF91F7
:102CD000CF911F910F91FF90EF90DF90CF900C94C8
:102CE000F925892F837009F079C001114BC2812F1A
:102CF000829586958770880F880F212F2F70C22E9E
:102D0000D12CE12CF12C082E04C0CC0CDD1CEE1CC7
:102D1000FF1C0A94D2F714FF12C04FE050E060E0AD
:102D200070E004C0440F551F661F771F8A95D2F7C5
:102D30008A019B01009510952095309503C000E015
:102D400010E09801969596959370492F50E0C9012F
:102D5000B80142305105D1F04330510559F16C2989
:102D60007D298E299F294130510541F127960FB6C3
:102D7000F894DEBF0FBECDBFDF91CF911F910F91B1
:102D8000FF90EF90DF90CF900C94EB1C6C297D2985
:102D90008E299F2927960FB6F894DEBF0FBECDBFB0
:102DA000DF91CF911F910F91FF90EF90DF90CF9027
:102DB0000C94FD1C0E94EB1CC701B60127960FB6B0
:102DC000F894DEBF0FBECDBFDF91CF911F910F9161
:102DD000FF90EF90DF90CF900C94D91C002319F056
:102DE000892F817001C08695882309F4CBC1812F7A
:102DF000829586958770880F880F212F2F70C22E9D
:102E0000D12CE12CF12C082E04C0CC0CDD1CEE1CC6
:102E1000FF1C0A94D2F714FF12C04FE050E060E0AC
:102E200070E004C0440F551F661F771F8A95D2F7C4
:102E30008A019B01009510952095309503C000E014
:102E400010E09801969596959370492F50E0C9012E
:102E5000B80142305105D1F04330510559F16C2988
:102E60007D298E299F294130510541F127960FB6C2
:102E7000F894DEBF0FBECDBFDF91CF911F910F91B0
:102E8000FF90EF90DF90CF900C94A21D6C297D29CC
:102E90008E299F2927960FB6F894DEBF0FBECDBFAF
:102EA000DF91CF911F910F91FF90EF90DF90CF9026
:102EB0000C94B41D0E94A21DC701B60127960FB63F
:102EC000F894DEBF0FBECDBFDF91CF911F910F9160
:102ED000FF90EF90DF90CF900C94901D103F41F148
:102EE00018F4103E48F48BC0123F09F450C0D8F1DA
:102EF000133F09F460C083C01F70892F8F710023B6
:102F000021F00E94291D812F7BCE0E944A1D812F16
:102F100027960FB6F894DEBF0FBECDBFDF91CF91DD
:102F20001F910F91FF90EF90DF90CF900C944F1571
:102F30000023A9F0253008F025C1892F8F7127962D
:102F40000FB6F894DEBF0FBECDBFDF91CF911F91BA
:102F50000F91FF90EF90DF90CF900C946F1D263073
:102F600008F010C1EACF0023A1F0892F8F712796B6
:102F70000FB6F894DEBF0FBECDBFDF91CF911F918A
:102F80000F91FF90EF90DF90CF900C94291D0023BC
:102F900061F3892F8F7127960FB6F894DEBF0FBEAD
:102FA000CDBFDF91CF911F910F91FF90EF90DF90F8
:102FB000CF900C944A1D002391F0892F8F71279692
:102FC0000FB6F894DEBF0FBECDBFDF91CF911F913A
:102FD0000F91FF90EF90DF90CF900C94141D2796E7
:102FE0000FB6F894DEBF0FBECDBFDF91CF911F911A
:102FF0000F91FF90EF90DF90CF900C940F1D002366
:10300000A1F0222309F4B1CF812F27960FB6F894AF
:10301000DEBF0FBECDBFDF91CF911F910F91FF900B
:10302000EF90DF90CF900C942614222309F4B1CFB7
:10303000812F27960FB6F894DEBF0FBECDBFDF916C
:10304000CF911F910F91FF90EF90DF90CF900C9454
:10305000F914492F4F70612FC6010E9483222796D1
:103060000FB6F894DEBF0FBECDBFDF91CF911F9199
:103070000F91FF90EF90DF90CF900C94211C0111E5
:1030800081C0112341F0892F8F70843021F0907F0F
:10309000212F2F70922B9F70892F90E08230910505
:1030A000E9F1ACF4009751F1019709F06BC0279654
:1030B0000FB6F894DEBF0FBECDBFDF91CF911F9149
:1030C0000F91FF90EF90DF90CF900C94992E83306A
:1030D0009105A1F1049709F055C0812F27960FB6ED
:1030E000F894DEBF0FBECDBFDF91CF911F910F913E
:1030F000FF90EF90DF90CF900C94302F27960FB673
:10310000F894DEBF0FBECDBFDF91CF911F910F911D
:10311000FF90EF90DF90CF900C946F2E27960FB614
:10312000F894DEBF0FBECDBFDF91CF911F910F91FD
:10313000FF90EF90DF90CF900C94C82E27960FB69B
:10314000F894DEBF0FBECDBFDF91CF911F910F91DD
:10315000FF90EF90DF90CF900C94FA2E492F4F7094
:10316000612FC60127960FB6F894DEBF0FBECDBF04
:10317000DF91CF911F910F91FF90EF90DF90CF9053
:103180000C94862227960FB6F894DEBF0FBECDBFF3
:10319000DF91CF911F910F91FF90EF90DF90CF9033
:1031A00008950E94A81F0E94771F0E94B91F0E94C5
:1031B0002B270E94F92580E090E00E94D61280E043
:1031C00090E00C94EC120E94981F0C94D1180E946D
:1031D000C71D292F22952F7030E02C3031054CF47B
:1031E0002A3031056CF4225031092230310588F43F
:1031F00007C02C30310549F02F30310531F009C0BE
:10320000803E48F0803F29F406C093FB882780F970
:10321000089580E0089581E00895CF93DF9300D072
:1032200000D01F92CDB7DEB70F900F900F900F9088
:103230000F90DF91CF910895CF93DF9300D000D00E
:1032400000D0CDB7DEB726960FB6F894DEBF0FBE1E
:10325000CDBFDF91CF9108951F93CF93DF93C0919E
:10326000C50316E08091C603C81799F0D0E01C9FF3
:10327000F0011D9FF00D1124E953FC4F4081518155
:1032800062817381848195810E941C192196C77087
:10329000E9CFDF91CF911F9108954091F7035091AD
:1032A000F8036091F9037091FA038091FB03909108
:1032B000FC030C941C198091FC0382958F7009F01B
:1032C00054C08091F903882309F44FC08091C5034D
:1032D000A091C6036091F7037091F8034091FA033F
:1032E0005091FB03B6E08A1709F43FC090E0411506
:1032F0005105C1F17F3F11F46F3FA1F1B89FF0017B
:10330000B99FF00D1124E953FC4F218172132AC09B
:103310002081621327C02281211124C0238134819E
:103320002417350710F421503109241B350B283C94
:103330003105C0F42091FC032F7020612093FC0321
:1033400026E0289FF001299FF00D1124E453FC4F43
:1033500080818F708061808387EF93E00E94561593
:103360000C942C1901968770BECF0895CF92DF92EE
:10337000EF92FF920F931F93CF93DF93CDB7DEB7FA
:1033800062970FB6F894DEBF0FBECDBF8C0185E00B
:10339000F801DE011D9601900D928A95E1F7D801A2
:1033A0004C9111965C91119712966C91129713960D
:1033B000CD90DC9014973091F7037091F8038091D1
:1033C000FA039091FB03009709F46BC17F3F19F456
:1033D0003F3F09F466C1E090F903EE2009F4C0C054
:1033E0002091FC03C816D90628F0F601E81BF90B5A
:1033F000CF0104C0809590958C0D9D1DFF24F39402
:10340000883C910578F0F12C207F09F0C6C07C2D16
:10341000D98AC88A89890E940D1987EF93E00E9492
:103420005615B1C0822F807F09F046C0751314C0B5
:10343000341312C0611110C02F7020612093FC035F
:103440000E944D1987EF93E00E9456158091FC036E
:10345000D80115968C932EC0CD2819F15F3F11F439
:103460004F3FF9F0F62E61111CC08091C5032091E9
:10347000C60336E0821709F45AC090E0389FF00185
:10348000399FF00D1124E953FC4F7181571306C089
:103490007081471303C07281711103C00196877058
:1034A000E9CFF62E662309F418C18091FC038160F0
:1034B0008093FC03F12C11C1751308C0341306C0AE
:1034C000611104C08091FC03D801C3C04D875E87A1
:1034D0008D859E856A8B0E94E7186A898823E1F1B1
:1034E0006623D1F12091FC03822F82958F7090E0AA
:1034F000029774F08091F7039091F80398878F8377
:103500001986DB86CA862C87CE0107960E9456153F
:1035100086E0F801A7EFB3E001900D928A95E1F7FC
:103520000E945B190E944D19FF24F394D6C04D8769
:103530005E878D859E850E94C71D292F22952F703D
:1035400030E0223031050CF0BCC09F7009F0B6C0ED
:10355000805E883008F4C1C0C8010E945615E4CFCF
:10356000C816D90608F453C0F601E81BF90BCF01C1
:10357000883C910508F450C0F12C7C2DD98AC88A6A
:1035800089890E940D19E7EFF3E086E0DF011D92C3
:103590008A95E9F70E944D19A0C0751314C0341321
:1035A00012C0611110C08091FC03F8018583C8012D
:1035B0000E94561586E0E7EFF3E0DF011D928A9541
:1035C000E9F7FE2C8AC04D875E878D859E856A8BC4
:1035D0000E94E7186A89882309F4BECF662309F49C
:1035E000BBCF2091FC03822F82958F7090E00297D1
:1035F0000CF48ECF8091F7039091F8039A8389831E
:103600001B82DD82CC822E83CE0101967FCF8095F6
:1036100090958C0D9D1DACCFF62E662309F49CCFA2
:1036200075132EC034132CC02091FC0320FD1FC045
:10363000822F82958F70D9F0D80115962C9315970B
:103640008F3049F08F5F982F9295907F822F8F70E7
:10365000892B15968C93C8010E94561586E0F801B7
:10366000A7EFB3E001900D928A95E1F793CF86E042
:10367000F801A7EFB3E001900D928A95E1F72DC014
:103680004D875E878D859E850E94E718811140CF0A
:103690008091FC0381608093FC03C8010E94561551
:1036A0001CC0662309F458CF4D875E878D859E85A3
:1036B0000E94E718882309F44FCF2ACF811148CF01
:1036C0000CC0243031050CF047CF9F7009F440CF77
:1036D000F8019581907F09F03BCF8F2D62960FB650
:1036E000F894DEBF0FBECDBFDF91CF911F910F9138
:1036F000FF90EF90DF90CF9008951F93CF93DF93CB
:10370000CDB7DEB72C970FB6F894DEBF0FBECDBF96
:103710004F83588769877A878B879C87CE01079666
:103720000E94B619882369F08F8198852A853B8588
:10373000232BF1F19F3F09F063C08F3F09F060C078
:1037400037C086E0FE013796DE01119601900D929A
:103750008A95E1F76F817885EA85FB85309741F19D
:103760007F3F11F46F3F21F12091C60330E0C90182
:103770000196877099274091C50350E084179507FB
:1037800009F447C069837A83FD83EC8396E0929FB6
:10379000D001939FB00D1124A953BC4FFE01319667
:1037A00001900D929A95E1F78093C6030E942C191F
:1037B00016E08091C5039091C6038917C1F1189F47
:1037C000C001112489539C4F0E94B619882379F1B6
:1037D000E091C5031E9FF0011124E953FC4F408185
:1037E000518162817381848195810E941C1980912D
:1037F000C50390E00196877099278093C503D9CFC0
:103800004F81588569857A858B859C850E941C1916
:10381000CFCF0E94E3181092C6031092C503E7EFC2
:10382000F3E086E0DF011D928A95E9F7C1CF2C967F
:103830000FB6F894DEBF0FBECDBFDF91CF911F91C1
:103840000895DF92EF92FF920F931F93CF93DF9330
:10385000FC01892B09F48AC0E12CF12CDD24D394DE
:10386000EF0121968491853709F461C058F48437BB
:1038700008F04EC0843008F06AC08130D1F0823048
:1038800071F174C0883709F45DC050F4863709F4CB
:1038900055C0873709F06AC08E2D0E94951F54C00D
:1038A0009CE7980F903708F061C08F770E94F91459
:1038B00050C08F010E5F1F4FFE01849190E2980F60
:1038C000983050F48770FD2D01C0FF0F8A95EAF7FC
:1038D0008F2F0E949B1F14C00E94261413C08F01BB
:1038E0000E5F1F4FFE01C49180E28C0F883060F4A0
:1038F000C7708D2D01C0880FCA95EAF70E94A11FDD
:103900000E94B91FE80125C08C2F0E94F914FACF3C
:103910009F012E5F3F4FFE01C491CC2369F08FE9D8
:103920009FE00197F1F700C00000C150F6CF9F0162
:103930002E5F3F4FFE01F490E9010BC00E94851FEE
:10394000E82E07C00E94981F0E94B91F02C00E9463
:1039500026148F2D882341F0EFE9FFE03197F1F72E
:1039600000C000008150F6CFFE017ACFDF91CF91E9
:103970001F910F91FF90EF90DF90089560930104E5
:103980007093020480930304909304040E945130C6
:103990000C94D1186093FD037093FE038093FF0392
:1039A000909300040E94B0300C94D11808950C94A8
:1039B000BE1C0F931F9300910104109102042091EB
:1039C000030430910404602B712B822B932B1F91E5
:1039D0000F910C94BE1C0F931F9300910104109142
:1039E0000204209103043091040460237123822394
:1039F00093231F910F910C94BE1C0F931F93009162
:103A00000104109102042091030430910404602702
:103A10007127822793271F910F910C94BE1C60E0A1
:103A200070E0CB010C94CA1C0F931F9341E050E04F
:103A300060E070E08A019B0104C0000F111F221F8B
:103A4000331F8A95D2F7C901B8011F910F910C94C9
:103A5000CA1C0F931F9341E050E060E070E004C087
:103A6000440F551F661F771F8A95D2F78091FD037B
:103A70009091FE03A091FF03B09100048A019B0185
:103A8000082B192B2A2B3B2BC901B8011F910F9131
:103A90000C94CA1C0F931F9341E050E060E070E06B
:103AA00004C0440F551F661F771F8A95D2F74095B3
:103AB0005095609570958091FD039091FE03A091C3
:103AC000FF03B09100048A019B01082319232A23D4
:103AD0003B23C901B8011F910F910C94CA1C0F938D
:103AE0001F9341E050E060E070E004C0440F551FB8
:103AF000661F771F8A95D2F78091FD039091FE0390
:103B0000A091FF03B09100048A019B0108271927A7
:103B10002A273B27C901B8011F910F910C94CA1C99
:103B20000F931F930091FD031091FE032091FF035B
:103B300030910004602B712B822B932B1F910F91DE
:103B40000C94CA1C0F931F930091FD031091FE0368
:103B50002091FF033091000460237123822393237B
:103B60001F910F910C94CA1C0F931F930091FD039A
:103B70001091FE032091FF0330910004602771270C
:103B8000822793271F910F910C94CA1C0895CF92FE
:103B9000DF92EF92FF920F931F93CF93DF938C01ED
:103BA000C0900104D0900204E0900304F09004045B
:103BB0004091FD035091FE036091FF03709100045A
:103BC000C42AD52AE62AF72ACFE1D0E0D701C601D8
:103BD0000C2E04C0B695A795979587950A94D2F7B1
:103BE00080FF07C0B8018C2F0E9410228130910500
:103BF00031F4219758F7B80180E00E941022DF913C
:103C0000CF911F910F91FF90EF90DF90CF9008958B
:103C1000CF92DF92EF92FF920F931F93CF93DF9398
:103C2000C82F80910A01882361F180910B018823BC
:103C300041F18C2F8695869586958F3088F4E0919A
:103C40000C01F0910D01E80FF11DC77081E090E0CB
:103C500001C0880FCA95EAF79181892B8183A3C09F
:103C600080911B0480FF9FC01F92CF938CEE92E047
:103C70009F938F930E94FB060F900F900F900F90D1
:103C800092C0D090180430911604E0910C01F0918C
:103C90000D01332309F473C0409117048D2D2FEFCC
:103CA00096E0E92EF12C082F082E000C110BBF0115
:103CB000600F711FDB0112969C919C1709F473C071
:103CC0002F3F19F4911101C0282FC801019606E079
:103CD00010E0B7010E94CA338413E5CFD22F4D11F3
:103CE0004EC02F3F69F4842F440F990B0196B80101
:103CF0000E94CA33809318043150309316043FC099
:103D0000822F220F990B0196B8010E94CA33282FE7
:103D1000FF24F39406E010E0022E000C330B6F0139
:103D2000C20ED31ED60112965C91552391F08D2FB1
:103D3000DD0F990BBF01680F791FDB0112965C93B1
:103D4000D60112961C920196B8010E94CA33D82F50
:103D500001C0F394C9010196B8010E94CA33282F0B
:103D60008413DACF242F440F330B2F193109C901E3
:103D7000069666E070E00E94CA3380931704809133
:103D80001704082E000C990BE80FF91FC283019647
:103D900066E070E00E94CA33809317048091160495
:103DA0008F5F80931604DF91CF911F910F91FF9049
:103DB000EF90DF90CF900895EF92FF920F931F93B3
:103DC000CF93DF93482F80910A01882369F1809176
:103DD0000B01882349F1842F8695869586958F302F
:103DE00090F4E0910C01F0910D01E80FF11D477086
:103DF00081E090E001C0880F4A95EAF780959181B3
:103E0000892381836DC080911B0480FF69C01F924C
:103E10004F938EEC92E09F938F930E94FB060F903E
:103E20000F900F900F905CC020911804E091160441
:103E3000EE2309F455C0C0910C01D0910D01009101
:103E40001704002E000C110B86E0E82EF12C30E058
:103E5000DE01A20FB31FCD01029612965C9154139E
:103E600035C0DC011C92E150E0931604E11104C05E
:103E7000109218041092170440911704842F042EF6
